:030000000219FDE5
:03000B000200AA46
:03002B0002015679
:03005B000202E9B5
:030073000202CFB7
:1000800002030406080C10182030406080040608A3
:100090000C10182030406080A0C000070F1F3F0DDB
:1000A0000D04050D050305030302C2AFC0D0C0E077
:1000B000206217E5256002E473E525F4F58A758B67
:1000C00000D262D0E0D0D0D2AF3285268AC262E5BB
:1000D00026F46035306803207210758B00D0E0D0B4
:1000E000D0D295D293D297D2AF32D295D293D29723
:1000F000206E0C206609740CD5E0FDE57E429075FB
:100100008B00D0E0D0D0D2AF32758A00C28DD262DF
:1001100001FF01B9306805206602C29501B9306857
:1001200005206602C29701B9306805206602C293B5
:1001300001B9C294306805206602C29501B9C29621
:10014000306805206602C29701B9C2923068052066
:100150006602C29301B9C2AFC2AD53E6EFC0D0C0D0
:10016000E0D2D3D2AFC2CEE52A6007207449152A67
:1001700021B77800790020742EE580307E01F430BC
:10018000E50278FF53DACF207E0343DA20307E0386
:1001900043DA10C2D8C271E580307E01F430E50246
:1001A00079FFC3E89970CB306103752A1820740376
:1001B000752A18885FD27020740DE52B6004152B0A
:1001C00021C743DA01C2D82070024125A85F20610F
:1001D00002C2702074367982B70431C3E894F040CB
:1001E0000374F0F8E8C4540F28F87984B703024187
:1001F0000CC313C3138721200802C313200A06C3AC
:10020000C898F8410C28F8500374FFF88822E52DAF
:1002100054066011E533C313C31324062522F522C7
:1002200050037522FF7882B60459852224A824C37E
:10023000E52495644002A864C3E895664002A86678
:100240008825E56970024176C3E8AA699A5003E8F7
:10025000FAE4F9EAC333FBE56BF45B29400D256A48
:10026000F8E56A6002156A400B41760AC3E56A9AAE
:100270005002056A78FF8826C26EC3E52694F840CE
:1002800002D26EC3E52594404002D26420CF0AD04A
:10029000E0D0D043E610D2AD32C2CF053A7801E5C6
:1002A0002A6005307402152AC3E55F940140057584
:1002B000620041C5756300756C00E5622401F5625A
:1002C00050037562FFD0E0D0D043E610D2AD32C209
:1002D000AFC0D053E67FC2607591008556948557B4
:1002E00095759104D0D0D2AF32C2AF53E6EFC2AD14
:1002F000C0D0C0E0C0F0D2D3D2AFA8FBA9FCC2D816
:10030000307102615053DACF207E0343DA10307E21
:100310000343DA20D271E580307E01F420E50261EA
:100320002788278928A17D53DACF207E0343DA204E
:10033000307E0343DA10C2D8C271307402A16978EA
:1003400000E580307E01F430E502A169885FA151AB
:1003500053DACF207E0343DA20307E0343DA10C223
:1003600071206102812953DACF207E0343DA1030F5
:100370007E0343DA20C2D8D271885A895BC3E895DC
:1003800058F8E99559F97B007E087A00C3E8948C07
:10039000E994005005755E00811B882178A2E6A8CB
:1003A000216055C3E894C8E994005008E4D2E4FB06
:1003B0007A0A61F6C3E89468E994015008E4D2E34C
:1003C000FB7A0F61F6C3E894D0E994025008E4D2B6
:1003D000E2FB7A1E61F6C3E894A0E994055008E4B4
:1003E000D2E1FB7A3C61F6C3E89498E9940850089E
:1003F000E4D2E0FB7A787E00C3E8955CFCE9955D89
:10040000FD30E70AECF42401FCEDF43400FD755EE8
:1004100000C3EC9AED9E5003755E01885C895D8592
:100420005A58855B597802A151C3E89527F8E99598
:1004300028F9307C02A135307B02A135307A02A147
:100440002E207502814CE9FDE8FC816BE9C313F9AC
:10045000E813F8307902A12EE9C313F9E813F83054
:100460007802A12EE9C313FDE813FC20612CC3EC34
:0E047000941CED940240028182ED701EC3ECDC
:10047E0094C850180529E52970021529C3E5299459
:10048E000A5002A169755F00D270A169E529600268
:10049E0015297888E6F97400207F087896B903024A
:1004AE00789EE624FAFEE43400FFC3EC9EFCED9F3A
:1004BE00FD9208B90310A2085007207609D2768162
:1004CE00D4307602C276A2085016B9030DECF4248D
:1004DE0001FCEDF43400FD0204EE78007900A13544
:1004EE00B90315EC33FCED33FDC3EC940AFCED942B
:1004FE0000FD50047C007D00C3EC94FFED940040A1
:10050E000678FF7900A135EC8575F0A4C5F0A2F749
:10051E0033F87900400302055178FF790002055146
:10052E00E9C313F9E813F8307C0EE9600278FFC3D3
:10053E00E81338F8E43400F9C3E894FFE994004076
:10054E000278FF885FD270206102A169741FF45592
:10055E002F4BF52FC274EB7002D274752A183074BB
:10056E0003752A0A306102A17D20740353DAFE203E
:10057E007403752B06D0F0D0E0D0D0D2AD43E61088
:10058E003279010205AD79030205AD790A0205AD96
:10059E00791E0205AD79640205AD79C80205AD7804
:1005AE0017E4D5E0FDD8FAD9F6227A147B78020545
:1005BE00D47A107B8C0205D47A0D7BB40205D47AE2
:1005CE000B7BC80205D47902B27DE4C296D5E0FD5C
:1005DE00C297D5E0FDD297D5E0FDD296D5E0FDC20B
:1005EE0095E576D5E0FDD2957496D5E0FDD9D9EA9C
:1005FE00F8D5E0FDD8FBDBCEC29622C37C007D0091
:10060E0075F00005F0EA33FAEB33FB50F6EB13FB13
:10061E00EA13FAC3E9FFE8FEE89AF8E99BF95004F9
:10062E00EFF9EEF8B3EC33FCED33FDD5F0DFEDF979
:10063E00ECF822E889F08A20D2D4F8A9F07B0030B9
:10064E00F70B7BFFF42401F8E9F43400F9E8852078
:10065E00F0A4ADF0F8E98520F0A4AFF0FEED2EF990
:10066E0074003FFA7C04C3EA13FAE913F9E813F8AD
:10067E00DCF48BF030F70AE8F42401F8E9F43400E6
:10068E00F9E889F0C2D4F8A9F0227882B604030200
:10069E0006F3C3E55F940140030206BD852224E400
:1006AE00F545F546F547F548F549C26D0206F3786E
:1006BE0082E6FCD26DE522F523783879C7AA40ABE5
:1006CE0041C3EB13FBEA13FAEC146013C3EB13FBF9
:1006DE00EA13FAEC14146007C3EB13FBEA13FAD116
:1006EE00098845894622C3E5459523F8E5469400D9
:1006FE00F9500CC3E89480E994FF4016020724C316
:10070E00E8947FE994005003020724787F79000271
:10071E000724788079FF884A894B22E54A2547F8D5
:10072E00E54B3548F9854B20E4300701F43549FA9D
:10073E0030E709C3EA94F04015020762C3EA940F4A
:10074E00500302076278FF79FF7A0F020762780082
:10075E0079007AF0C3E5249564500AC37401952498
:10076E00500B020780E54B20E70E020780E54B3069
:10077E00E706884789488A492278A4E6FAC3E54AFB
:10078E0033F8E54B33F9D141E930E70BC3E89480F8
:10079E00E994FF4013E1BAC3E8947FE99400500254
:1007AE00E1BA787F7900E1BA788079FFE820E71521
:1007BE00C3E52398F84009C3E8940140030207E11A
:1007CE0078010207E1E8F424012523F8400302072B
:1007DE00E178FF884C2278A5E6FAA848A949D141CC
:1007EE00E930E70CC3E89401E994FF4016020815BE
:1007FE00C3E894FFE99400500302081578FF7900CE
:10080E00020815780179FFE920E715C3E54C98F841
:10081E004009C3E89401400302083C780102083CF9
:10082E00E8F42401254CF8400302083C78FF8824A4
:10083E002278FFC26420693D206A12D264C3E5416A
:10084E00940A4009C3E52594405002C26479A1E799
:10085E006023E541601F74FF8541F0848539F030D7
:0F086E006A0375F005A4F8C5F0600278FFC3E8CF
:10087D0095675002A867886622C3E5409440E5411C
:10088D009401E5665003140197046002F566220297
:10089D00089F2275E890227883E6FFE5E820ECF7C3
:1008AD00A8BDA9BE0573C3E57394084052757300C6
:1008BD00E9FA79A0E76044EA7007E574601B020865
:1008CD00DAC3E895746010E5745006600C140208E4
:1008DD00E60460F90208E6E574F574C3946D401BF7
:1008ED007564C0C394044013756480C39404400BB5
:1008FD00756440C39404400375640075BB0822E51C
:10090D00642410500274FFF5647982B70402213318
:10091D00C3A864E524985002A824C3E89566400254
:10092D00A86688258826E573B4070375BB10227465
:10093D003279A687F0A4C5F0A2F733F8C3E8956421
:10094D004002A86488228824882588268867227515
:10095D0040007541F022C2AF75C820A8CCA9CDAA20
:10096D003A30CF010A75C824D2AFAB3BAC3C883BC3
:10097D00893CC3E89BF8E99C206908F9306702417E
:10098D007821D5AD3D8A3DF9EA9DFA600478FF796D
:10099D00FFAE3EAF3F8B3E8C3FC3EC9FFCC3E99C4B
:1009AD00F542A83BA93CC3E89EF8E99FF9C3E54190
:1009BD0013FBE54013FAE82AF540E93BF5415006F3
:1009CD007540FF7541FF411FAA40AB41AC40AD41A1
:1009DD007E047F02C3EB940440021E1FC3EB9408F8
:1009ED0040021E1FC3ED13FDEC13FCDEF7C3EA9CA2
:1009FD00FAEB9DFBEF6009C3E913F9E813F8DFF794
:100A0D00EA28FAEB39FB8A408B4150067BFF8B407D
:100A1D008B41C3EB94025002D2673069047F0341CE
:100A2D004A7892E6FFC3E537948240110FC3E5374C
:100A3D0094A040010FC3EF940640027F057E05E5AB
:100A4D0041C4540FF9E541C454F0F8E540C4540FC6
:100A5D0028F8C3E89EFAE99400FB4009C3EA940222
:100A6D00EB940050047A02E4FB41C4AA40AB41EB85
:100A7D00C4FEEAC4540F4EFCC3EA9CFAEB9400FB8F
:100A8D00C3E813C313F8EA28FAEB3400FB8A408B52
:100A9D0041C3EB94024002C2677805EBC4FE7B00B4
:100AAD00EAC4540F4EFAC3EA98FA4005C3940250B3
:100ABD00027A027892E6FF30600241C48552568573
:100ACD005357D26043E680C3E49AF8E49BF930674C
:100ADD0002615EE8FAE9FBD3E913FDE813FC8852E5
:100AED008953C3EF94036038EF20E00DE82CF8E94B
:100AFD003DF9ECFAEDFB020B19E828F8E939F9C3D9
:100B0D00E82402F8E93400F97AFE7BFFC3EF940381
:100B1D00400E8A548B55884E894F8C508D51619261
:100B2D00885489558A4E8B4F8C508D51306920C316
:100B3D00E53394034019E542A2E713F8E555F42493
:100B4D000138400B20E7087554FFF42401F5556179
:100B5D0092E8FAD3E813FC8852C3EF94036020EFB8
:100B6D0020E007E82CF8ECFA617EE8282402F87AF8
:100B7D00FEC3EF940340088A54884E8C50619288CE
:100B8D00548A4E8C50E56BC3335002646BF56B3059
:100B9D006002619C753402D26043E680E52D5406F7
:100BAD006026A840A941C3E913F9E813F8C2AF5371
:100BBD00E67F759100C3E498F594E499F5957591E8
:100BCD0004D26043E680D2AF22D265754400752011
:100BDD0000306B03752040020BF5D265754400752E
:100BED002040306B03752000D2AF7801206722E5DD
:100BFD002D54066002C265C3E54194054013780289
:100C0D00940540087803940540027806306902780F
:100C1D000A206019E544601530690AC3E533940371
:100C2D004003D53406D2AFD26C81C671A4D2AF00C9
:100C3D0000C2AF206726E541C3FB940F40027B0F36
:100C4D00EB240530730123306A02742820620123DE
:100C5D00F93069027982E58BC39940B50544E59B6E
:0F0C6D005440B5200281B030690A08C3E8940AE8
:100C7C00400108811E20650261F5C26553E67F754F
:100C8C0091003067107594007595FE759104D260D3
:100C9C0043E68061F5AE40AF41C3E49EF594E49F1A
:100CAC00F5958197C3E5339402500261F5306502E6
:100CBC0061F5D80281C4811EC26C53E67F75910028
:100CCC00855494855595759104854E56854F57D20C
:100CDC006043E680D2AFE52D54066008206A020519
:100CEC0033020D00306C0D206B0A20650715811541
:100CFC008102156B2278003064053065027801E5BD
:100D0C003775F007A4F9E5F028F5F0E9A2F013A285
:100D1C00F113A2F213F537C394785003753778C3E7
:100D2C00E53795384008D266D295D293D297306089
:100D3C0002A13A855056855157D26043E680222055
:100D4C007D11C2AF754302C296D294D2AF759F117A
:100D5C00020F1AC2AF754302C296D292D2AF759FE0
:100D6C0011020F1A307243207D20C2AF75430390DD
:100D7C00013E757E40D293C292306204C297A18E1E
:100D8C00D296D2AF759F13020F1AC2AF7543039060
:100D9C00013E757E40D295C294306204C297A1AEDA
:100DAC00D296D2AF759F10020F1A207D17C2AF7565
:100DBC00430390011ED293306202C297D2AF759F4B
:100DCC0013020F1AC2AF75430390011ED295306205
:100DDC0002C297D2AF759F10020F1A207D11C2AFBD
:100DEC00754304C294D292D2AF759F10020F1AC2EF
:100DFC00AF754304C292D294D2AF759F13020F1AEF
:100E0C00307243207D20C2AF754305900132757E50
:100E1C0010D297C296306204C295C12AD294D2AF36
:100E2C00759F11020F1AC2AF75430590014A757E6A
:100E3C0004D297C296306204C293C14AD292D2AF06
:100E4C00759F11020F1A207D17C2AF7543059001D3
:100E5C0014D297306202C295D2AF759F11020F1A4D
:100E6C00C2AF754305900128D2973062EBC293D282
:100E7C00AF759F11020F1A207D11C2AF754306C2C8
:100E8C0092D296D2AF759F13020F1AC2AF7543065A
:100E9C00C294D296D2AF759F10020F1A30724220B4
:100EAC007D20C2AF75430190014A757E04D295C274
:100EBC0094306204C293C1C6D292D2AF759F100215
:100ECC000F1AC2AF754301900132757E10D293C2D6
:100EDC0092306204C295C1E6D294D2AF759F13E1F1
:100EEC001A207D16C2AF754301900128D29530624D
:100EFC0002C293D2AF759F10E11AC2AF7543019035
:100F0C000114D293306202C295D2AF759F13C266A0
:100F1C0022900112757E00D295D293D297C294C2C0
:100F2C0092C296C262227880760908760908760405
:100F3C000876FF0876030876FF08760A0876030819
:100F4C007601087601788C76010876FF0876FF0822
:100F5C0076FF0876FF0876FF0876030876FF08769A
:100F6C00FF0876FF0876250876D008762808765094
:100F7C000876040876FF08760208760008767A0868
:100F8C0076FF087601087601087600087603227849
:100F9C0087E6FFC272BF0302D2727888E6C394035D
:100FAC006008C27DE630E102D27DC27E7889E630EF
:100FBC00E102D27EC3EF94026008758E01D27302F7
:100FCC000FD3758E00C273227880E6149000809344
:100FDC0078A4F67881E6149000809378A5F678864C
:100FEC00E61490008D9378A6F6789CE67538FF751C
:100FFC00390CB402067538A075390AB40306753875
:10100C008275390578A3E61490009A93F569120F4E
:10101C001D22227896E6FA7897E6FB7888E6B403E8
:10102C0005C3EB940EFB307F047A007BFFC3EB9A75
:10103C00FCC3948250027C827575000575EC857535
:10104C00F0A4C3E5F0947D40F222D27F111F12056B
:10105C009E7A007B007C10120594E55F2AFA7400DE
:0F106C003BFBDCF37C04C3EB13FBEA13FADCF76A
:10107B00FEC27F111F22E5EF20E60375200005203D
:10108B00903FFFE520146006901DFF146000930451
:10109B00600375EF1253D9BF7581C043FF801205F2
:1010AB008F75EF0243B203E5B3240420E70DF5215E
:1010BB00E5E320E0068521B343E301120F1D7580A4
:1010CB00FF75A40075F1B275D4DF7590A975A5FCF9
:1010DB0075F2FE75D50175A60175E241E4F8F6D8F7
:1010EB00FD756B01120F321215AD7898867675303F
:1010FB0001C2AF1205A81205B812059E1205BF1248
:10110B00059E1205C612059EC2AF78FA79FA308594
:10111B0007D9FBD8F7021C00120F9B120FD4111E1C
:10112B00111F78988676120F1D7588507589127568
:10113B00C82475910475D84075A82275B80275E658
:10114B0090759B80759D0075D10E75BC5875BB084D
:10115B0075BA1175E88012058FD2AF12089C53DA5D
:10116B00CF207E0343DA20307E0343DA1043DA01CB
:10117B00C2D8C2711205A8D2617B037A0CE55E70EE
:10118B00077A0CDB0302111312059E207003021168
:10119B0013C270E55FC3940240E1E52F541F8561D4
:1011AB0060F561B560D5DAD5C26153DACF207E0325
:1011BB0043DA20307E0343DA10C2D8C27178A2E63C
:1011CB007008D274E52F54E0F52FC2757529001203
:1011DB0005A3307409C3E529940A4002D2751205A0
:1011EB009478023074027800C3E55F9840F0C2AF88
:1011FB001205B81205B81205B8D2AF1205A8754D75
:10120B00007888E6B4030241EA120594788CE6C3B1
:10121B00940150030212EAE530C394015003021209
:10122B00EA207435C3E55F94FF50030212EAC2AFA4
:10123B001205CDD2AF1205A3C3E55F940150EFC2E7
:10124B00AF1205B81205991205B8D2AF1205A3C398
:10125B00E55F94FF40E90217557F02D27F111F1201
:10126B0005A3C2AFC27F111FAE5FC3E55F947FD2F0
:10127B00AF407612058FC2AF1205CDD2AFDFDC11B6
:10128B0056C3EE94057897F61205A81215EF1216B1
:10129B00D87F0AD27F111F1205A3C2AFC27F111FC5
:1012AB00AE5FC3E55F947FD2AF50E612058FC2AF3E
:1012BB001205B81205991205B8D2AFDFD61156EE4A
:1012CB0024057896F61205A81215EF1217071205CA
:1012DB00A3111FC3E55F94FF5002412C021755C3A6
:1012EB00E55F954D4003855F4D1205A37801798825
:1012FB00E7B403027805C3E55F984002410CC2AF27
:10130B001205CD1205CD1205CDD2AF1205A8753041
:10131B0000E4F531F5320531E531F47039053278F9
:10132B009AE67819146012783214600D787D146087
:10133B000878FA146003753200C3E532984017152C
:10134B00327531B478998676C2AF1205CDD2AF78AB
:10135B009886761205A3120599E52A70053074025A
:10136B00211378012074027806C3E55F9840A778B3
:10137B0088E6C3940360031205A3E52A70030211E8
:10138B0013C2AF120F1DE4F522F523F524F525F555
:10139B0026F56AD2AF7885E6C333F568E4F545F5F3
:1013AB0046F547F548F549F573F52CF52DF53775E9
:1013BB00730875BB1012058F1208A0E5E820ECFB33
:1013CB00A8BDA9BEE97001F888741208A47573084A
:1013DB0075BB107887E6FE7602120F9B7887EEF6C8
:1013EB00C2AF7564FF12093C852264852265852294
:1013FB0066D2AF752201752401752501752601850D
:10140B00636C756D017888E6B40307C27D30760294
:10141B00D27DD268D269753300120E83120EA812D8
:10142B00095C12096312095C12096312095C02144C
:10143B0049C2AF120F9BD2AF75730075BB08120B6D
:10144B00E7120698120D01120D4B120963120BD6FF
:10145B00306D031206F420670312083F3067031246
:0E146B000886120D01120D70120963120BE7B4
:10147900306D03120729120D01120DE712096312CB
:101489000BD6306D03120787120D01120E0C1209CB
:1014990063120BE7306D031207E4120D01120E837C
:1014A9001209631208A0120BD6120D01120EA8120E
:1014B90008A4120963306935206B32856764856732
:1014C9006585636C756D0179187A0CC3E5339940AC
:1014D9000FC269D26A8A358567648567660214F620
:1014E900C3E55F94014003021449021573306A1B76
:1014F900206B18E535147004C26A813CF535C3E5E3
:101509005F94014003021449021573753600C3E55F
:101519006278FA985054307404E52A604D7888E668
:10152900B40317207D05207607A143307602A14335
:10153900206B07D26B856764818878F0306B0585ED
:1015490067647820C3E5419850028149306B1BC21A
:101559006BC27D307602D27DD26A75351285676499
:1015690081490536E55F6002A176753600C2AF1282
:101579000F1D7887E6FE7602120F9B7887EEF6E458
:10158900F522F523F524F525F526F568C268D2AFCD
:1015990012058F120F1D307409C3E53694054002F8
:1015A9002113611C901A0D7820121631E520B455CB
:1015B9000CA3121631E520B4AA030215CF120F327B
:1015C9001215EF0215EE901A0378807B0A12163174
:1015D900A308DBF9901A0F788C7B18121631A3082F
:1015E900DBF9901A2722C2AF12167012164A901A06
:1015F90000740E121636A37404121636A37414124C
:101609001636901A0378807B0A121635A308DBF97F
:10161900901A0F788C7B18121635A308DBF912166D
:1016290083121661901A2722E493F622E6438F016A
:10163900538FFD75EF0275B7A575B7F1F0538FFE9E
:1016490022438F02438F0175EF0275B7A575B7F174
:10165900901A0DF0538FFC22901A0D7455D13690C3
:101669001A0E74AAD136227A3079D07820901A408D
:10167900D131E520F709A3DAF7227A3079D0901A27
:1016890040E7D13609A3DAF922AB77A878BB010282
:101699007980BB02027981BB03027982BB0402799A
:1016A90084BB05027986BB06027992BB070279875A
:1016B900BB080279A3BB0902799CBB0A027988BBE2
:1016C9000B027989E8F7227C051205A8DCFB22C206
:1016D900AF1205B81205BF1205C61205CD1205993C
:1016E9001205B81205BF1205C61205CD12059912C9
:1016F90005B81205BF1205C61205CDD2AF22C2AF79
:101709001205CD1205C61205BF1205B812059912A8
:1017190005CD1205C61205BF1205B81205991205A5
:10172900CD1205C61205BF1205B8D2AF22AE77AFEA
:1017390078C2AF1205B81205B81205B8120599DEBC
:10174900F21205CD120599DFF8D2AF22D1D8D1D046
:10175900D1D0757701757801757900F1367C05ADC1
:101769005F1205A8C3ED955F70F5C3E55F9401406D
:101779000AC3E55F94FF4032021791D192B1EFD1CC
:10178900D8C2AF75EF12D1D0DCD50579C3E579940C
:1017990003500280C6D1D00578E5771490009F9355
:1017A900F808C3E57898500280AED1D0D1D005773A
:1017B900C3E577940C5002809C120F32B1EFC2AF8F
:0517C90075EF12D1D004
:0319FD0002108154
:101A00000E0414090904FF03FF0A03010155AA018A
:101A1000FFFFFFFFFF03FFFFFF25D0285004FF0259
:081A2000007AFF01010003FF41
:101A400023526F746F724765656B73323041232088
:101A500023424C48454C4923463333302320202031
:101A60002020202020202020202020202020202076
:101C0000C2AFC2D353D9BF7581C043B20343FF8073
:101C1000752438752503B1C975EF0275E24043F1AB
:101C20002053A4DF75D400D2857DFA780379E67C51
:101C300010752200752300901DD67B0675249875BB
:101C400025013085028142208508D8FBD9F9DCF7CF
:101C500081B4308508D8FBD9F9DCF781B4B189E4C7
:101C600093A3C39A6004DDC381B4DBDBB17B600264
:101C7000812B7B08E493FAA3B15CDBF87A30B15C8A
:101C8000752200752300B17BEAFCEBFDC3ED94FEE9
:101C9000400EB17B8A278B28ED30E0048A828B834B
:101CA000B17B7AC270D8C3ED94FE601350CEBD00F4
:101CB00025EC60097520007521FF0200008100A855
:101CC00027A9280809D804D90281D3B17FEA89AAB3
:101CD000F281C50D81A0C3ED94035049EDA2E092BD
:101CE000007AC5C3E5829400E583941C50902000DF
:101CF00010438F02438F0175B7A575B7F1F030001F
:101D00001FA827A9280809438F01538FFDD804D99C
:101D100002A12089AAE275B7A575B7F1F0A3A10DBC
:101D2000538FFC817C7AC1BD030CE493A3FAB140CC
:101D3000DCF8B138817C817EAA22AB23B15CEBFA5E
:101D4000EA6222752608C3E52313F523E52213F57D
:101D50002250066323A0632201D526EAB1C9B1C986
:101D600075260AEAF4200102D285300102C285B14B
:101D7000C9C3134002C201D526EB22B17FEAFB2082
:101D80008502A17F308502A184752608AE24AF2587
:101D9000C3EF13FFEE13FEB1CDB1C9C3EA13308513
:101DA000024480FA30E703632201C3E52313F523DD
:101DB000E52213F52250066323A0632201D526D91C
:101DC000E52265236523F52222AE24AF250E0FDE22
:101DD000FEDFFCD20122424C48656C693437316326
:041DE000F3300601D5
:00000001FF
